:020000040800F2
:1000000000040020A1020008A3020008A3020008C7
:10001000A3020008A3020008A3020008A30200082C
:10002000A3020008A3020008A3020008A9260008F2
:10003000A3020008A3020008A3020008A30200080C
:10004000A3020008A3020008A3020008A3020008FC
:10005000A3020008A3020008ED3B0008193C0008B9
:10006000453C0008713C00089D3C0008A3020008C4
:10007000A3020008A3020008A3020008A3020008CC
:10008000A3020008A3020008A3020008A3020008BC
:10009000A3020008A3020008A3020008C93C00084C
:1000A000A3020008A3020008A3020008A30200089C
:1000B000A3020008A3020008A3020008A30200088C
:1000C000A3020008A3020008A3020008A30200087C
:1000D000A3020008A3020008A3020008A30200086C
:1000E000313D0008A3020008A3020008A302000893
:1000F000A3020008A3020008A3020008A30200084C
:10010000A3020008A30200086D380008A30200083B
:10011000A3020008A3020008A3020008A30200082B
:10012000A3020008A3020008A3020008A30200081B
:10013000A3020008A3020008A3020008A30200080B
:10014000A3020008A3020008A3020008A3020008FB
:10015000A3020008A3020008A3020008A3020008EB
:10016000A3020008A3020008A3020008A3020008DB
:10017000A3020008E1310008A3020008A30200085E
:10018000A3020008A3020008A50F0008A3020008AC
:10019000A3020008A3020008A3020008A3020008AB
:1001A000A3020008A3020008A3020008A30200089B
:1001B000A3020008A3020008A3020008A30200088B
:1001C000A3020008A3020008A3020008A30200087B
:1001D000A3020008CD310008A3020008A302000812
:1001E000A3020008A3020008A3020008A30200085B
:1001F000A3020008A3020008A3020008A30200084B
:10020000A3020008A3020008A3020008A30200083A
:10021000A3020008A3020008A3020008A30200082A
:10022000A3020008A3020008A3020008A30200081A
:10023000A3020008A3020008A3020008A30200080A
:10024000A3020008A3020008A3020008A3020008FA
:10025000A3020008A3020008A3020008A3020008EA
:10026000A3020008A3020008A3020008A3020008DA
:10027000A3020008A3020008A3020008A3020008CA
:10028000A3020008A3020008A3020008A3020008BA
:10029000A3020008A3020008A3020008A3020008AA
:1002A00002E000F000F8FEE772B6394880F30888F3
:1002B000384880F3098838484EF60851CEF20001DC
:1002C000086040F20000CCF200004EF63471CEF22D
:1002D00000010860BFF34F8FBFF36F8F40F2000043
:1002E000C0F2F0004EF68851CEF200010860BFF374
:1002F0004F8FBFF36F8F4FF00000E1EE100A4EF604
:100300003C71CEF200010860062080F31488BFF330
:100310006F8F02F007FA03F027FA4FF055301F49AC
:100320001B4A91423CBF41F8040BFAE71C49194AA9
:1003300091423CBF41F8040BFAE71A491A4A1B4B99
:100340009A423EBF51F8040B42F8040BF8E7002034
:100350001749184A91423CBF41F8040BFAE702F0F2
:1003600025FA03F075FA144C144DAC4203DA54F834
:10037000041B8847F9E700F03FF8114C114DAC42DF
:1003800003DA54F8041B8847F9E702F00DBA0000BD
:1003900000040020002400200000000800000020CD
:1003A0000004002088410008002400203824002098
:1003B0003824002050390020A0020008A0020008C4
:1003C000A0020008A00200082DE9F04F2DED108AD0
:1003D000C1F80CD0D0F80CD0BDEC108ABDE8F08F7D
:1003E000002383F311882846A047002001F000FE77
:1003F00001F0B0FD00DFFEE738B5204C6FF074036C
:10040000002523701E236570A570E5702571657148
:10041000A571E57125726572A372E57200F0E8FCC2
:1004200020B10E2325726572A372E57202F00CF9F9
:10043000044602F033F90546D8B9114B9C421AD054
:1004400001339C4218BF054641F2883404BF0125A0
:100450000024002002F0FEF80DB100F0B7F800F023
:1004600031FD00F049FC204600F070F900F0AEF8D4
:10047000F9E70024EDE70446EBE700BF382400204D
:10048000010007B008B500F0B5FBA0F12003584209
:10049000584108BD07B5054B02211B88ADF8043053
:1004A00001A800F013FC03B05DF804FB503E000807
:1004B000064991F8243033B100230822086A81F8F4
:1004C000243000F03DBC0120704700BF58240020BC
:1004D0002DE9F84F234C94F82430054688461746FA
:1004E0008BBB2E46DFF87C90002F38D094F824A0E8
:1004F000BAF1000F05D12022FF214846266200F004
:10050000CFFCCAF10805BD4228BF3D465FFA85FB16
:10051000AD0041462A4604EB8A0000F097FC94F8AF
:100520002430A7EB0B079B445FFA8BFBBBF1080F52
:100530002E44A844FFB284F824B0D5D1FFF7B8FF09
:100540000028D1D108E0266A06EB8306B042C9D064
:10055000FFF7AEFF0028C4D10020BDE8F88F0120CE
:10056000BDE8F88F5824002010B5202383F31188AC
:100570001248C3680BB101F0C1FD0023104A0F48B7
:100580004FF47A7101F07EFD002383F311880D4C46
:10059000236813B12368013B2360636813B1636868
:1005A000013B6360084B1B7833B9636823B90220B1
:1005B00000F03AFC3223636010BD00BF44240020E9
:1005C0006905000888290020802400202DE9F041D9
:1005D000544B554953F8042F013201D1BDE8F08145
:1005E0008B42F7D1514C524B22689A4240F298808C
:1005F000504B9B6803F1006303F500339A4280F08F
:100600008F80002000F094FB4B4B0220187000F00C
:10061000FFFB4A4BD3F8E8200022C3F8E820D3F8C8
:100620001011C3F81021D3F81011D3F8EC10C3F84F
:10063000EC20D3F81411C3F81421D3F81411D3F813
:10064000F010C3F8F020D3F81811C3F81821D3F82C
:100650001811D3F8801041F00061C3F88010D3F86E
:10066000801021F00061C3F88010D3F88010D3F817
:10067000801041F00071C3F88010D3F8801021F091
:100680000071C3F88010D3F8803072B62C492D4B1E
:100690000B601D682468BFF34F8FBFF36F8F2A4B29
:1006A000C3F88420BFF34F8F5A6922F480325A6115
:1006B000BFF34F8FD3F88020C2F3C906C2F34E3286
:1006C0005201B70743F6E07E02EA0E08384631468B
:1006D000013948EA000CB1F1FF3FC3F874C200F1E0
:1006E0004040F5D1203A12F1200FEDD1BFF34F8FEA
:1006F000BFF36F8FBFF34F8FBFF36F8F5A6922F431
:1007000000325A610022C3F85022BFF34F8FBFF36B
:100710006F8F202383F31188AD4685F30888204727
:10072000BDE8F081FCFF01081C000208040002087B
:10073000FFFF0108382400208024002000440258D4
:1007400008ED00E00000020800ED00E02DE9F04FA8
:10075000B54C97B020228246FF210EA8A56800F074
:100760009FFBB24A1378A046A3B9B1480121C360E8
:100770001170202383F31188C3680BB101F0BEFC14
:100780000023AC4AAA484FF47A7101F07BFC0023A5
:1007900083F31188DFF8BCB2BAF1000F01D0CBF8B7
:1007A00000A0A54F00243C70CBF804402646012051
:1007B00000F02EFBBAF1000F00F0E081DBF8003012
:1007C000002B40F0DB8117B0BDE8F08F0220FFF76F
:1007D00059FE002840F0D081984B1B88ADF824309A
:1007E000022109A800F072FAE1E74FF47A7000F0F4
:1007F00001FA031E0193EFDB0220FFF743FE81465F
:100800000028E9D0019B581E0428E5D8DFE800F055
:10081000030C0F12150016A8052340F8343D0421DF
:1008200000F054FA4C4650E004217F48F8E70421D8
:100830008348F5E704218348F2E71C24204600F0B2
:1008400079FA04340990042109A800F03FFA2C2C0D
:10085000F4D1E7E7002EBFD0002CBDD00220FFF777
:1008600011FE064610B901242646B5E7012000F026
:100870005FFA0220387000F0CBFA0024E3B2184689
:10088000019300F065FA814648B1019B184600F0DB
:100890006FFA01340028F1D134466B4B9DE70123F8
:1008A00002203B7000F0A6FA4D46D8F808309D4271
:1008B00006D2284600F03EFA0130EDD10435F4E7C7
:1008C00000253D70CBF80450344600F0F1FAFFF7F4
:1008D000E1FD4EE1002E3FF47FAF002C3FF47CAFF2
:1008E0000220387000F094FA322000F083F9041EE0
:1008F000B9DB14F00306B6D1D8F808202B199342BF
:10090000B1D8B4F5807FAED8DFF84091A6420CDABA
:100910004FF47A7000F06EF90390039B002BA2DB7A
:10092000039B06F809300136F0E7C820FFF7AAFD5F
:100930000646002897D01F2D11D8C5F12009A145E2
:1009400028BFA1460EAB25F003004A463F49184494
:1009500000F07CFA4A46FF213C4800F0A1FA4FEA39
:10096000A4095FFA89F239492846FFF7B1FD044628
:10097000002891D005EB89050646A6E70220FFF77F
:1009800081FD00283FF428AFFFF792FD00283FF4D7
:1009900023AF4FF0000AD146D8F808309A453CD230
:1009A000BAF11F0F1CD80E9B013319D02AF0030394
:1009B00016AA134453F8203C099325494B68A3B168
:1009C000002209A8135C83EA0903DBB2013251F863
:1009D0002330042A83EA1929F4D10AF1040ADBE757
:1009E000504600F0A7F90990E7E71A46082012F0F0
:1009F000010F4FEA52021FBF82F06D4282F43802AB
:100A000082F4034282F020020138F0D141F8232021
:100A10000133B3F5807FE8D1D2E716A8042140F86E
:100A2000489D00F053F950E7382400208425002029
:100A3000442400206905000880240020523E00085C
:100A40003C24002040240020543E00088424002040
:100A5000882500208829002016A8002340F8343D6E
:100A6000642100F0FFF800287FF4B6AE0220FFF703
:100A700009FD00283FF4B0AE099800F08BF916ABE1
:100A800043F8440D04211846CBE716A8002340F88C
:100A9000343D642100F0E6F800287FF49DAE02208A
:100AA000FFF7F0FC00283FF497AE099800F074F9C6
:100AB00016AB43F8400DE5E70220FFF7E3FC002802
:100AC0003FF48AAE00F06EF916AB43F83C0DD9E75F
:100AD0000220FFF7D7FC00283FF47EAE09A91420BE
:100AE00000F066F9814616A8042140F8389D00F010
:100AF000EDF8494609A894E74FF47A70FFF7C2FC75
:100B000000283FF469AEFFF7D3FC00283FF4C5AEE0
:100B10000E9B01330CD008220EA90020FFF7D8FC51
:100B200000283FF4BAAE2022FF210EA800F0B8F949
:100B3000FFF7B0FC2E4801F061FA44E616A8002346
:100B400040F8343D642100F08DF800287FF444AE75
:100B50000220FFF797FC00283FF43EAEFFF79AFC17
:100B600041F2883001F04AFA099800F0E7F900F004
:100B70009FF94FF0000A1AE60646A6E6002000F0AC
:100B800039F80390039B002BFFF614AE012000F010
:100B900031F9039B213B122B3FF609AE01A252F81B
:100BA00023F000BFCD070008EB0700085508000838
:100BB000AF070008AF070008AF070008D508000816
:100BC000AF0700087D090008590A00088B0A0008D1
:100BD000B90A0008AF070008D10A0008AF070008EB
:100BE000F90A0008CB080008AF0700083D0B000811
:100BF000A08601002DE9F34702AE00244FF47A7578
:100C000006F8014D144FDFF85880454397F900303E
:100C10005A1C5FFA84F901D0A34212D158F824007B
:100C200003680122D3F820A031462B46D047012883
:100C300007D10A4B9DF8070083F8009002B0BDE889
:100C4000F0870134022CE1D14FF4FA7001F0D6F9AB
:100C50004FF0FF30F2E700BF00240020AC29002055
:100C6000583E00082DE9F0474FF47A75144FDFF82D
:100C7000588006464D43002497F900305A1C5FFA0D
:100C800084F901D0A34210D158F82400036804224B
:100C9000D3F820A031462B46D047042805D1094B74
:100CA00083F800900020BDE8F0870134022CE3D1E6
:100CB0004FF4FA7001F0A2F94FF0FF30BDE8F08771
:100CC00000240020AC290020583E000830B4074B17
:100CD0001A78074B53F822402368DD69054B0A4612
:100CE000AC460146204630BC604700BFAC2900201E
:100CF000583E0008A0860100F8B501F0C1FB094C80
:100D0000094E0A4F2070002530682378834207D9A6
:100D100001F0B2FB336805440133BD423360F3D9BF
:100D2000F8BD00BFAD29002090290020FFFF010081
:100D300001F076BC00F1006000F5003000687047FB
:100D400000F10060920000F5003001F003BC0000EB
:100D5000054B1A68054B1B789B1A834202D9104435
:100D600001F08ABB0020704790290020AD290020A7
:100D700038B5074D04462868204401F083FB28B9A4
:100D800028682044BDE8384001F08EBB38BD00BF64
:100D90009029002000207047014BC058704700BFC9
:100DA00000E8F11F014B1868704700BF0010005C9D
:100DB00070B50E4B5C6893F9086001380A18013C65
:100DC0000B4693420FD214F9015F581C1DB1034624
:100DD00000F8015CF5E72C2482421C7001D9981CB4
:100DE0005E70401A70BD1846FBE700BF0424002067
:100DF00000207047022804D14FF40002034B9A618F
:100E000070470128FCD14FF48002F7E70008025830
:100E1000022803D18022034B9A6170470128FCD13C
:100E20004022F8E700080258022805D1064A536913
:100E300083F08003536170470128FCD1024A536953
:100E400083F04003F6E700BF0008025810B5002306
:100E5000934203D0CC5CC4540133F9E710BD0000C9
:100E600030B5441E14F9010F0B4660B193F90050E0
:100E7000854201F1010106D11AB993F90020801AC7
:100E800030BD013AEEE7002AF7D1104630BD000030
:100E900002460346981A13F9011B0029FAD170473C
:100EA00002440346934202D003F8011BFAE770475D
:100EB000024B1A78024B1A70704700BFAC29002011
:100EC0000024002038B5174D174C284600F0C8FB09
:100ED0002146284600F0F0FB23681448D3F8902000
:100EE000D2F8043843F00203C2F8043801F086F85F
:100EF0000F49206800F0F0FC23680E48D3F89020DA
:100F00000D49D2F8043823F00203C2F80438A8428D
:100F10004FF4E1330B6003D0BDE8384000F0FEBA77
:100F200038BD00BF5C2E00202C3F000840420F005F
:100F3000743F0008B02900209429002038B50B4BDD
:100F40001A780B4B53F822400A4B9C4205460CD0B2
:100F5000094B002118461822FFF7A2FF0560014641
:100F60002046BDE8384000F0D9BA38BDAC29002091
:100F7000583E00085C2E002094290020024A136885
:100F800043F0C0031360704700780040044B5A6878
:100F900010439A6858600AB1181D1047704700BF87
:100FA000B02900202DE9F84F404EF56D2F68EC690F
:100FB0002C62210718D014F0080F0CBF00208020ED
:100FC000E20748BF40F02000A30748BF40F04000C0
:100FD000610748BF40F48070202383F31188FFF736
:100FE000D5FF002383F31188E20509D5202383F37D
:100FF00011884FF40070FFF7C9FF002383F31188B5
:10100000DFF8A8A04FF020094FF0000B14F02008E3
:1010100032D13B0615D5DFF898A04FF02009200605
:101020000FD589F31188504600F0ECF9002830DA2A
:101030000820FFF7ABFF27F080032B60002383F32A
:10104000118879060DD562060BD5202383F311880C
:10105000F26C336D9A4201D1336C03BB002383F3EE
:101060001188E30604D5B26E13690BB15069984735
:10107000BDE8F84F01F028BB89F31188AB8C96F8D6
:1010800064105046194000F057FA8BF31188EC6950
:10109000BCE780B2288588F31188EC69BFE710208F
:1010A00027F04007FFF772FF2F60D7E7B029002035
:1010B000E829002013B5104C204600F023FA04F173
:1010C0001400009400234FF400720C4900F0E4F87F
:1010D00004F1380000940A4B0A494FF4007200F002
:1010E0005DF9094BE365094B23660C21522002B0E0
:1010F000BDE8104000F05EB8B02900201C2A002096
:101100007D0F00081C2C00200078004000E1F50550
:10111000254B002908BF1946037C8166012B30B599
:1011200011D1224B98420ED1214BD3F8E82042F046
:101130008042C3F8E820D3F8102142F08042C3F87F
:101140001021D3F810310A68036EC46D03EB52030B
:10115000B3FBF2F34A68150442BF23F0070503F01E
:10116000070343EA4503E3608B6843F04003636091
:10117000CB6843F00103A36042F4967343F001038C
:10118000236051054FF0FF33236205D512F0102282
:1011900005D0B2F1805F04D080F8643030BD7F2389
:1011A000FAE73F23F8E700BF703E0008B0290020AF
:1011B0000044025800F1604300F01F02400903F5AB
:1011C000614309018000C9B200F1604083F8001357
:1011D00000F5614001239340C0F8803103607047FF
:1011E000F8B5154682680669AA420B46816938BF80
:1011F0008568761AB542044607D218462A46FFF794
:1012000025FEA3692B44A3610DE011D9324618468F
:10121000FFF71CFEAF1B3A46E1683044FFF716FEAD
:10122000E2683A44A261A3685B1BA3602846F8BD4C
:1012300018462A46FFF70AFEE368E4E783682DE9CB
:10124000F041044693421546266938BF85684069D7
:10125000361AB5420F4606D22A46FFF7F7FD6369F4
:101260002B4463610DE012D93246A5EB0608FFF767
:10127000EDFD4246B919E068FFF7E8FDE268424437
:101280006261A3685B1BA3602846BDE8F0812A4623
:10129000FFF7DCFDE368E4E710B50A440024C3610E
:1012A000029B006040608460C160816141610261B5
:1012B000036210BD08B582694369934201D1826817
:1012C00082B98268013282605A1C42611970426997
:1012D00003699A4201D3C3684361002100F0AAFE6A
:1012E000002008BD4FF0FF3008BD000070B520237E
:1012F00004460E4683F31188A568A5B1A368A269C8
:10130000013BA360531CA36115782269934224BF5B
:10131000E368A361E3690BB120469847002383F398
:101320001188284670BD3146204600F073FE002823
:10133000E2DA85F3118870BD2DE9F74F05460F46B7
:1013400090469A46D0F81C90202686F311884FF0DC
:10135000000B144664B1224639462846FFF740FF89
:10136000034668B95146284600F054FE0028F1D0E3
:10137000002383F31188A8EB040003B0BDE8F08FCD
:10138000B9F1000F03D001902846C847019B8BF3A9
:101390001188E41A1F4486F31188DBE7C16081617C
:1013A0004161C3611144009B006040608260016143
:1013B00003627047F8B504460E461746202383F3B0
:1013C0001188A568A5B1A368013BA36063695A1C95
:1013D00062611E70236962699A4224BFE368636197
:1013E000E3690BB120469847002080F31188F8BDCF
:1013F0003946204600F00EFE0028E2DA85F3118817
:10140000F8BD0000836942699A4210B501D1826833
:101410007AB98268013282605A1C82611C78036941
:101420009A4201D3C3688361002100F003FE204685
:1014300010BD4FF0FF3010BD2DE9F74F05460F46A8
:1014400090469A46D0F81C90202686F311884FF0DB
:10145000000B144664B1224639462846FFF7EEFEDB
:10146000034668B95146284600F0D4FD0028F1D063
:10147000002383F31188A8EB040003B0BDE8F08FCC
:10148000B9F1000F03D001902846C847019B8BF3A8
:101490001188E41A1F4486F31188DBE70268436869
:1014A0001143016003B11847704700001430FFF783
:1014B00043BF00004FF0FF331430FFF73DBF000083
:1014C0003830FFF7B9BF00004FF0FF333830FFF777
:1014D000B3BF00001430FFF709BF00004FF0FF3129
:1014E0001430FFF703BF00003830FFF763BF000080
:1014F0004FF0FF323830FFF75DBF0000002070472B
:10150000FFF7D8BD044B0360002343608360C360D2
:1015100001230374704700BF883E000810B52023E4
:10152000044683F31188FFF7F3FD0223237400239D
:1015300083F3118810BD000038B5C36904460D4619
:101540001BB904210844FFF7A9FF294604F1140040
:10155000FFF7B0FE002806DA201D4FF48061BDE8D9
:101560003840FFF79BBF38BD0268436811430160F4
:1015700003B118477047000013B5446BD4F8943496
:101580001A681178042915D1217C022912D1197900
:10159000128901238B4013420CD101A904F14C00A4
:1015A00001F050FFD4F89444019B21790246206851
:1015B00000F0EAF902B010BD143001F0D3BE000013
:1015C0004FF0FF33143001F0CDBE00004C3001F07D
:1015D000A5BF00004FF0FF334C3001F09FBF00006B
:1015E000143001F0A1BE00004FF0FF31143001F0C3
:1015F0009BBE00004C3001F071BF00004FF0FF3285
:101600004C3001F06BBF0000D0F8942438B513685B
:1016100019780429054601D0012038BD017C022932
:10162000FAD112795C89012090400440F4D105F18F
:10163000140001F033FE02460028EDD0D5F8945492
:101640004FF480732868697900F08CF9204638BD22
:10165000406BFFF7D9BF00000020704770470000C3
:101660007FB5124B0360002343608360C360012594
:1016700002260F4B057404460290019300F1840288
:10168000294600964FF48073143001F0E3FD094BB6
:101690000193029400964FF4807304F52372294657
:1016A00004F14C0001F0AAFE04B070BDB03E000889
:1016B00051160008791500080A68202383F3118861
:1016C0000B790B3342F823004B79133342F8230094
:1016D0008B7913B10B3342F8230002230374C0F853
:1016E0009414002383F311887047000038B5037FFA
:1016F000044613B190F85430ABB9201D01250221E6
:10170000FFF732FF04F1140025776FF0010100F0BC
:101710009DFC84F8545004F14C006FF00101BDE8C9
:10172000384000F093BC38BD10B5012104460430A8
:10173000FFF71AFF0023237784F8543010BD000010
:1017400038B504460025143001F09CFD04F14C002E
:10175000257701F06BFE201D84F854500121FFF71E
:1017600003FF2046BDE83840FFF74EBF90F88030B9
:1017700003F06003202B19D190F88120212A0AD090
:10178000222A4FF000030ED0202A0FD1084A4267C8
:101790000722826704E0064B436707238367002321
:1017A000C3670120704743678367F9E700207047EC
:1017B00010240020D0F8943437B51A681178042921
:1017C00004461AD1017C022917D119791289012303
:1017D0008B40134211D100F14C05284601F0E6FE82
:1017E00058B101A9284601F02DFED4F89444019B7C
:1017F00021790246206800F0C7F803B030BD000030
:1018000001F10B03F7B550F8234005460E46F4B13D
:10181000202383F3118805EB8607201D0821FFF79D
:10182000A3FEFB685B691B684C3413B1204601F0D2
:1018300017FE01A9204601F005FE024648B1019BB2
:101840003146284600F0A0F8002383F3118803B046
:10185000F0BDFB685A691268002AF5D01B8A013B6B
:101860001340F1D105F18002EAE70000133138B5E9
:1018700050F82140DCB1202383F31188D4F894245C
:101880001368527903EB8203DB689B695D6845B19D
:1018900004216018FFF768FE294604F1140001F0E6
:1018A00007FD2046FFF7B0FE002383F3118838BD03
:1018B0007047000001F002B8012303700023436069
:1018C00000F1300200F1500142F8043B8A42D3613A
:1018D000FAD103814381704738B50446202383F34E
:1018E00011880025416000F10C0300F1300243F83B
:1018F000045B9342FBD1204601F002F802232370DF
:1019000085F3118838BD000070B500EB81030546F2
:101910005069DA600E46144618B110220021FFF714
:10192000BFFAA06918B110220021FFF7B9FA3146B9
:101930002846BDE8704001F0F5B80000038903F0C7
:1019400001030381438903F00103438100F1300265
:1019500000F11003002143F8041B9342FBD101F076
:1019600079B90000F0B400EB81044789E4680125EF
:10197000A4698D403D43458123600023A2606360DC
:10198000F0BC01F095B90000F0B400EB81040789C8
:10199000E468012564698D403D430581236000238F
:1019A000A2606360F0BC01F00DBA0000022310B524
:1019B000037000230446A0F8883080F88A3080F84D
:1019C0008B300381438100F10C0200F1300142F8B9
:1019D000043B8A42FBD184F87030204601F036F88F
:1019E00063681B6823B120460021BDE810401847FA
:1019F00010BD0000436802781B6880F88C20052227
:101A000002700BB10421184770470000436890F83A
:101A10008C201B6802700BB105211847704700002D
:101A200090F8703070B5044613B1002380F8703020
:101A300004F18002204601F031F963689B6863BBC2
:101A400094F8805015F0600615D194F8813005F0B7
:101A50007F0545EA032540F202339D4200F00E81E6
:101A60005BD8022D00F0DC803FD8002D00F087808D
:101A7000012D00F0CF800021204601F0C7FB00219E
:101A8000204601F0B7FB63681B6813B106212046AE
:101A90009847062384F8703070BD20469847002888
:101AA000CED094F8872094F8863043EA0223A26FC0
:101AB000934238BFA36794F98030A56F002B4FF095
:101AC000200380F2FD80002D00F0EC80092284F8D4
:101AD000702083F311880021A36F626F2046FFF707
:101AE00053FF002383F3118870BDB5F5817F00F0AB
:101AF000B180B5F5407F49D0B5F5807FBBD194F872
:101B00008230012BB7D1B4F8883023F00203A4F857
:101B100088306667A667E667C3E740F201639D42C7
:101B20001ED8B5F5C06F3BD2B5F5A06FA3D1B4F800
:101B30008030B3F5A06F0ED194F8823084F88A30EB
:101B4000204600F0E1FF63681B6813B101212046C5
:101B500098470323237000236367A367E367A0E725
:101B6000B5F5106F32D040F602439D4252D0B5F524
:101B7000006F80D104F18B036367012324E004F13B
:101B8000880363670223A367E5678AE794F88230D6
:101B9000012B7FF470AFB4F8883043F00203B6E74E
:101BA00094F88520616894F884304D6894F8831027
:101BB00043EA0223204694F88220A84700283FF4F5
:101BC0005AAF436863670368A367A4E72378042BCD
:101BD00010D1202383F311882046FFF7AFFE86F350
:101BE0001188636884F88B601B68032121700BB136
:101BF0002046984794F88230002BACD084F88B3084
:101C00000423237063681B68002BA4D002212046A4
:101C10009847A0E7374B63670223A36700239DE73C
:101C200094F8841011F0800F204601F00F010ED0BF
:101C300001F026F8012806D002287FF41CAF2E4BB5
:101C40006367A06767E72D4B6367A56763E701F0EC
:101C500009F8EFE794F88230002B7FF40CAF94F88A
:101C6000843013F00F013FF476AF1A06204602D5F8
:101C700001F0E4FA6FE701F0D5FA6CE794F88230EE
:101C8000002B7FF4F8AE94F8843013F00F013FF48A
:101C900062AF1B06204602D501F0B8FA5BE701F0FF
:101CA000A9FA58E7142284F8702083F311882B4690
:101CB0002A4629462046FFF755FE85F3118870BD58
:101CC0005DB1152284F8702083F311880021A36F81
:101CD000626F2046FFF746FE03E70B2284F8702070
:101CE00083F311882B462A4629462046FFF74CFEEF
:101CF000E3E700BFE03E0008D83E0008DC3E0008F5
:101D000038B590F870300446152B29D8DFE803F079
:101D10003E28282828283E28280B29392828282822
:101D2000282828283E3E90F8871090F88620836F58
:101D300042EA01229A4214D9C268128AB3FBF2F530
:101D400002FB15356DB9202383F311882B462A46F3
:101D50002946FFF719FE85F311880A2384F87030AD
:101D600038BD142384F87030202383F311880023B6
:101D70001A4619462046FFF7F5FD002383F3118824
:101D800038BDC36F03B198470023E7E7002101F096
:101D90003DFA0021204601F02DFA63681B6813B15B
:101DA0000621204698470623D8E7000090F87020C7
:101DB000152A38B5044622D80123934040F64162E3
:101DC00013421DD113F480150FD19B0217D50B239D
:101DD00080F87030202383F311882B462A46294649
:101DE000FFF7D2FD85F3118838BDC3689B695B6836
:101DF0002BB9C36F03B19847002384F8703038BD06
:101E0000002101F003FA0021204601F0F3F9636894
:101E10001B6813B10621204698470623EDE7000012
:101E2000024B00221B605B609A6070471C2E0020F2
:101E3000002303748268054B1B6899689142FBD2AA
:101E40005A68036042601060586070471C2E002082
:101E500008B5202383F31188037C032B05D0042BC2
:101E60000DD02BB983F3118808BD436900221A6095
:101E70004FF0FF334361FFF7DBFF0023F2E790E809
:101E80000C001A6002685360F2E70000002303743C
:101E90008268054B1B6899689142FBD85A680360B9
:101EA00042601060586070471C2E0020054B196975
:101EB0000874186802681A6053601861012303747B
:101EC000FEF782BA1C2E002030B54B1C87B00546A9
:101ED0000A4C10D023690A4A01A800F0D3F828461A
:101EE000FFF7E4FF049B13B101A800F007F9236991
:101EF000586907B030BDFFF7D9FFF8E71C2E002066
:101F0000511E000838B50C4D41612B6981689A68F3
:101F10009142044603D8BDE83840FFF789BF184610
:101F2000FFF786FF01232C61014623742046BDE89C
:101F30003840FEF749BA00BF1C2E0020044B1A6837
:101F40001B6990689B68984294BF002001207047ED
:101F50001C2E002010B5084C236820691A682260E6
:101F60005460012223611A74FFF790FF0146206933
:101F7000BDE81040FEF728BA1C2E00208260022225
:101F800002740022427470478368A3F17C0243F814
:101F90000C2C026943F83C2C426943F8382C074A60
:101FA00043F81C2CC26843F8102C022203F8082CBA
:101FB000002203F8072CA3F118007047E103000882
:101FC00010B5202383F31188FFF7DEFF00210446BC
:101FD000FFF798FF002383F31188204610BD00000F
:101FE000024B1B6958610F20FFF760BF1C2E0020B9
:101FF000202383F31188FFF7F3BF000008B50146E3
:10200000202383F311880820FFF75EFF002383F36A
:10201000118808BD49B1064B42681B6918605A60B7
:10202000136043600420FFF74FBF4FF0FF3070474D
:102030001C2E00200368984206D01A680260506087
:1020400059611846FFF7F4BE7047000038B50446E2
:102050000D462068844200D138BD036823605C606F
:102060004561FFF7E5FEF4E7054B03F114025A6101
:102070009A614FF0FF32DA6100221A62704700BFA6
:102080001C2E0020F8B503611A4BC2605C6A1A4B23
:102090001A46022952F8145F38BF022195420646BB
:1020A0001F460AD1586198611C62056045608160D5
:1020B0000819BDE8F84001F09BBA186AAB68241A09
:1020C0000C1902D3E41A2D6804E09C4202D2204489
:1020D00001F09EFAAB689C42F4D86B68736035607F
:1020E0001E606E60B460A9684FF0FF33091BA960E1
:1020F000FB61F8BD000C00401C2E002010B41A4CEF
:10210000234653F8141F814210D0416802680A60C8
:10211000026851609A424FF00001C16003D0936899
:1021200081680B4493605DF8044B70470A686261F4
:1021300000209A425360C86003D15DF8044B01F05F
:1021400061BA9368886803449360084A206A526AB7
:10215000121A9342E7D9991A012998BF931C18447F
:102160005DF8044B01F054BA1C2E0020000C004016
:1021700000207047FEE70000704700004FF0FF307E
:1021800070470000022906D0032906D0012906481D
:1021900018BF0020704705487047032A9ABF0448BB
:1021A00000EBC20000207047D03F0008843F0008C9
:1021B0001824002070B5044608460D46FEF768FE58
:1021C000C6B22046013403780BB9184670BD3246BA
:1021D0002946FEF745FE0028F3D1012070BD00001E
:1021E0002DE9F04F80469BB008460C461646FEF798
:1021F0004FFE3A49C5B22046FFF7DCFF08B1013572
:10220000EDB237492046FFF7D5FF08B11035EDB2E2
:10221000632D01AF0CD8DFF8D490DFF8D4A03D4691
:1022200094F800B0BBF1000F1CD185F800B003E0BA
:102230002146384601F004FE3846FEF729FEC0B2BA
:10224000431C5B0088E8480033700323737000234D
:1022500002361946DAB2904206F1020636D81BB0B1
:10226000BDE8F08FBBF1250F2BD107221B4920467B
:10227000FEF7F6FD40B9DAF800302B60DAF80430EA
:102280006B6007340835CBE7082215492046FEF776
:10229000E7FDB0B91349AB1C11F8012F100902F08A
:1022A0000F0210F8090012F8092003F8012C0E4A59
:1022B00003F8020C914203F10203EDD11835083402
:1022C000AEE785F800B001340135A9E7FA5C06F8FD
:1022D000022C06F8011C0133BCE700BF343F0008A4
:1022E0003C3F0008FFE7F11F0BE8F11F4E3F0008DD
:1022F000453F000808B5202383F311880348FFF702
:1023000059FA002383F3118808BD00BF5C2E00201A
:1023100010B50446052916D8DFE801F01615031696
:10232000161D202383F311880E4A0121FFF7ECFAD2
:1023300020460D4A0221FFF7E7FA0C48FFF700FAA2
:10234000002383F3118810BD202383F311880748ED
:10235000FFF7CCF9F4E7202383F311880348FFF754
:10236000E3F9EDE7E43E0008083F00085C2E00209A
:1023700038B50C4D0C4C0D492A4604F10800FFF706
:102380002FFF05F1CA0204F110000949FFF728FFE9
:1023900005F5CA7204F118000649BDE83840FFF798
:1023A0001FBF00BF2433002018240020603F000816
:1023B000683F00083C3F0008BFF34F8F044B1A6989
:1023C0005107FCD1D3F810215207F8D1704700BF54
:1023D0000020005208B50D4B1B78ABB9FFF7ECFF9E
:1023E0000B4BDA68D10741BF0A4A5A6002F18832C2
:1023F0005A60D3F80C21D20741BF064AC3F8042122
:1024000002F18832C3F8042108BD00BF82350020E4
:10241000002000522301674508B5114B1B78F3B922
:10242000104B1A69510742BFDA6842F04002DA6085
:10243000D3F81021520742BFD3F80C2142F04002DA
:10244000C3F80C21FFF7B8FF064BDA6842F001022F
:10245000DA60D3F80C2142F00102C3F80C2108BD68
:1024600082350020002000520F289ABF00F58060BE
:1024700040040020704700004FF400307047000017
:10248000102070470F2808B50BD8FFF7EDFF00F5B7
:1024900000330268013204D104308342F9D10120B3
:1024A00008BD002008BD00000F2810B504464AD81A
:1024B000FFF782FFFFF78EFF24484FF0FF33072C12
:1024C0004361C0F8143124D80361FFF775FF23027C
:1024D00043F02403C360C36843F08003C36003690F
:1024E0005A07FCD4FFF768FF2046FFF7BDFF00F551
:1024F0000033BFF34F8F164A984220D3BFF34F8F5C
:10250000BFF36F8FFFF788FF2046BDE81040FFF74D
:10251000B9BFC0F81031FFF74FFFA4F108031B0249
:1025200043F02403C0F80C31D0F80C3143F08003A1
:10253000C0F80C31D0F810315B07FBD4D2E7C2F8F9
:102540005C022030D8E7002010BD00BF0020005200
:1025500000ED00E02DE9F84F42EA0003DB060646F5
:10256000884691464AD1FFF735FFDFF8B0B04546BF
:10257000A9EB050343441F2B04D8FFF74DFF0120AF
:10258000BDE8F88F204A2148214F06F17843934255
:10259000204B214A98BF9A4603F1FC0386BF1F4691
:1025A00092465846FFF708FF4FF0FF3303603B6841
:1025B00043F002033B6005F11C022B1FA6EB050E46
:1025C000DAF8004014F00504FAD153F8041F4EF86D
:1025D00003109342F4D1BFF34F8FFFF7EDFE4FF09E
:1025E000FF3303603B6823F002033B60202229464F
:1025F000304601F015FC20B1FFF70EFF0020BDE8CA
:10260000F88F20362035B3E7FFFF0F00142100526A
:102610000C200052102000521021005214200052B1
:1026200010B5084C237828B153B9FFF7D3FE012326
:10263000237010BD23B12070BDE81040FFF7ECBE41
:1026400010BD00BF82350020014B186D704700BFE0
:1026500000400058084B1A6F120405D41A6F1A670D
:102660001A6F42F400421A67044A136843F48073F5
:102670001360034B18657047004402580048025825
:1026800000400058034B1B685B0142BF024B012214
:102690001A707047D044025883350020014B1878D7
:1026A000704700BF83350020064A536823F00103BA
:1026B0005360EFF30983683383F30988002383F3BE
:1026C0001188704730EF00E010B5202383F31188A4
:1026D000104B5B6813F4006318D0F1EE103AEFF37F
:1026E00009844FF0807344F84C3C0B4BDB6844F892
:1026F000083CA4F1680383F30988FFF71FFC18B1B5
:10270000064B44F8503C10BD054BFAE783F31188A3
:1027100010BD00BF00ED00E030EF00E0F103000865
:10272000F4030008F0B5BFF34F8FBFF36F8F1D4B5D
:102730000021C3F85012BFF34F8FBFF36F8F5A6958
:1027400042F400325A61BFF34F8FBFF36F8FC3F86B
:102750008410BFF34F8FD3F88020C2F3C904C2F3B3
:102760004E325201A50743F6E07602EA060E2846ED
:1027700021464EEA00070139C3F860724F1C00F190
:102780004040F6D1203A12F1200FEED1BFF34F8F27
:102790005A6942F480325A61BFF34F8FBFF36F8F93
:1027A000F0BD00BF00ED00E0FEE70000084A094B65
:1027B00009498B4204D3094A0021934205D370474B
:1027C00052F8040F43F8040BF3E743F8041BF4E753
:1027D000BC410008503900205039002050390020F9
:1027E000D0F8943030B500229D68D0F89040114662
:1027F0004FF0FF3004EB421301329542C3F8001949
:10280000C3F81019C3F80809C3F8001BC3F8101B5C
:10281000C3F8080BEED24FF00113C4F81C3830BDDA
:1028200000EB81032DE9F04FD3F80CE0DEF8144003
:102830004F1CD4F800C03F034FEA41186568D0F838
:10284000902065450AD3D2F83438012000FA01F10E
:1028500023EA0101C2F83418BDE8F08FBEF8106019
:10286000ACEB0503B34228BF334602EB0806D6F8AB
:102870001869B6B2B3EB860F13D8A6683A44A6F12E
:10288000040A99465AF804BFC2F800B0B9F1040F1F
:1028900002D9A9F10409F5E71E442B44A660636040
:1028A000CCE70020BDE8F08F890141F020010161F3
:1028B00003699B06FCD4122000F03CBF10B50A4C03
:1028C0002046FEF7F9FF094BC4F89030084BC4F8D6
:1028D0009430084C2046FEF7EFFF074BC4F89030C9
:1028E000064BC4F8943010BD843500200000084029
:1028F000144000082036002000000440204000085A
:102900000378012B70B505465DD1494BD0F8904056
:10291000984259D1474BD3F8D82042F00062C3F80F
:10292000D820D3F8002142F00062C3F80021D3F888
:102930000021D3F8802042F00062C3F88020D3F851
:10294000802022F00062C3F88020D3F880300E216E
:102950006520FEF72FFC384BE360384BC4F8003895
:102960000023C4F8003EC0232360D5F890604FF4E4
:102970000413A3633369002BFCDA012333610C20B9
:1029800000F0D8FE3369DB07FCD4122000F0D2FE41
:102990003369002BFCDA0026A6602846FFF720FFEB
:1029A0006B68C4F81068DB68C4F81468C4F81C6865
:1029B000002B3AD1224BA3614FF0FF336361A36830
:1029C00043F00103A36070BD1E4B9842C8D1194B60
:1029D000D3F8D82042F00072C3F8D820D3F80021F1
:1029E00042F00072C3F80021D3F80021D3F8802010
:1029F00042F00072C3F88020D3F8802022F00072E9
:102A0000C3F88020D3F88020D3F8D82022F0806249
:102A1000C3F8D820D3F8002122F08062C3F8002147
:102A2000D3F800310E214D2093E7074BC3E700BFD9
:102A30008435002000440258401400400300200266
:102A4000003C30C020360020083C30C0F8B5D0F83B
:102A50009040054600212046FFF726FFD5F8941048
:102A600000234FF001128F68C4F834384FF000662D
:102A7000C4F81C284FF0FF3004EB431201339F428F
:102A8000C2F80069C2F8006BC2F80809C2F8080B66
:102A9000F2D20B68D5F89020C5F898306362102305
:102AA0001361166916F01006FBD1122000F042FEE9
:102AB000D4F8003823F4FE63C4F80038A36943F463
:102AC000402343F01003A3610923C4F81038C4F86D
:102AD00014380B4BEB604FF0C043C4F8103B094B6C
:102AE000C4F8003BC4F81069C4F80039D5F8983030
:102AF00003F1100243F48013C5F89820A362F8BDD7
:102B0000F03F000840800010D0F8902090F88A1024
:102B1000D2F8003823F4FE6343EA0113C2F8003808
:102B2000704700002DE9F0410EB200EB86080D461B
:102B3000D8F80C100F6807F00303022B53D0032BB7
:102B400053D03F4A3F4F012B18BF1746D0F8904053
:102B50004FEA451E04EB0E030022C3F8102B8A69CE
:102B600005F1100C002A42D04A8A05F158035B0196
:102B70003A43E2500123D4F81C2803FA0CF3134320
:102B8000A6444A69C4F81C380023CEF8103905F170
:102B90003F03002A3BD00A8A898B9208012988BF0B
:102BA0004A43D0F8981004EB8303561841EA0242D6
:102BB000C0F8986029465A602046FFF775FED8F89D
:102BC0000C301B8A43EA85531F4305F148035B0120
:102BD000E7500123D4F81C2803FA05F51543C4F87F
:102BE0001C58BDE8F081184FB0E7184FAEE704EB72
:102BF0004613D3F8002B22F40042C3F8002BD4F87C
:102C00001C28012303FA0CF322EA0303B8E704EBC0
:102C100083030F4A5A6004EB461629462046FFF705
:102C200043FED6F8003923F40043C6F80039D4F83F
:102C30001C38012202FA05F523EA0505CFE700BF9B
:102C400000800010008004100080081000800C102C
:102C500000040002D0F894201268C0F89820FFF712
:102C6000BFBD00005831D0F8903049015B5813F4D3
:102C7000004004D013F4001F14BF0120022070474D
:102C80004831D0F8903049015B5813F4004004D02B
:102C900013F4001F14BF01200220704700EB8101D4
:102CA000CB68196A0B6813604B685360704700006B
:102CB00000EB810330B5DD68AA691368D36019B9E8
:102CC000402B84BF402313606B8A1468D0F8902097
:102CD0001C44013CB4FBF3F46343033323F00303CC
:102CE00002EB411043EAC44343F0C043C0F8103B39
:102CF0002B6803F00303012B09B20ED1D2F8083878
:102D000002EB411013F4807FD0F8003B14BF43F076
:102D1000805343F00053C0F8003B02EB4112D2F85D
:102D2000003B43F00443C2F8003B30BD2DE9F041C5
:102D3000D0F8906006EB41130546D3F8087BC3F842
:102D4000087B3A070C4608D5D6F814381B0704D57B
:102D500000EB8103DB685B689847FA072FD5D6F84C
:102D60001438DB072BD505EB8403D968CCB98B6904
:102D7000488A5E68B6FBF0F200FB12628AB91868F6
:102D8000DA6890420DD2121A83E81400202383F3EC
:102D9000118821462846FFF78BFF84F31188BDE890
:102DA000F081012303FA04F26B8923EA02036B81A9
:102DB000CB6823B121462846BDE8F0411847BDE85D
:102DC000F081000000EB810370B5DD68D0F8903031
:102DD0006C692668E6604A0156BB1A444FF400202D
:102DE000C2F810092A6802F00302012A0AB20ED1C1
:102DF000D3F8080803EB421410F4807FD4F80009DC
:102E000014BF40F0805040F00050C4F8000903EBBC
:102E10004212D2F8000940F00440C2F80009D3F889
:102E20003408012202FA01F10143C3F8341870BDDD
:102E300019B9402E84BF4020206020682E8A841952
:102E400040F00050013C1A44B4FBF6F440EAC440A0
:102E5000C6E700002DE9F041D0F8906006EB411381
:102E60000446D3F80879C3F80879FB070D461CD54A
:102E7000D6F81038DA0718D500EB8103D3F80CE048
:102E8000DEF81430D3F800C0DA6894451BD2A2EB08
:102E90000C024FF000081A60C3F80480202383F36B
:102EA0001188FFF78FFF88F311883B0618D5D6F8F5
:102EB00034280123AB40134212D029462046BDE8F6
:102EC000F041FFF7ADBC012303FA01F2038923EAC5
:102ED00002030381DEF80830002BE6D09847E4E7D0
:102EE000BDE8F0812DE9F047D0F890506E69AB69EC
:102EF0001E40F10404466E6103D5BDE8F047FEF7BD
:102F000055BD002E11DAD5F8003E9A071EBFD5F840
:102F1000003E23F00303C5F8003ED5F8043823F043
:102F20000103C5F80438FEF771FD330502D52046CC
:102F3000FEF760FDB7040CD5D5F8083813F0060F7E
:102F4000EB6823F470530CBF43F4105343F4A053C5
:102F5000EB60300704D56368DB680BB12046984707
:102F6000F10200F1A180B2020BD5D4F890800027C5
:102F70004FF00109D4F894309B68F9B28B4280F08D
:102F8000D280F3061AD5D4F890100A6AC2F30A1751
:102F900002F00F0302F4F012B2F5802F00F0EC8083
:102FA000B2F5402F0AD104EB830301F58051DB68B1
:102FB000186A00231A469F4240F0D1803003D5F8AA
:102FC000185835D5E90303D500212046FFF7AEFE9A
:102FD000AA0303D501212046FFF7A8FE6B0303D502
:102FE00002212046FFF7A2FE2F0303D5032120462E
:102FF000FFF79CFEE80203D504212046FFF796FE6A
:10300000A90203D505212046FFF790FE6A0203D5E9
:1030100006212046FFF78AFE2B0203D50721204612
:10302000FFF784FEEF0103D508212046FFF77EFE5F
:10303000700340F1C980E90703D500212046FFF75E
:1030400009FFAA0703D501212046FFF703FF6B07FD
:1030500003D502212046FFF7FDFE2F0703D50321EC
:103060002046FFF7F7FEEE0603D504212046FFF7C2
:10307000F1FEA80603D505212046FFF7EBFE690601
:1030800003D506212046FFF7E5FE2A0603D50721D2
:103090002046FFF7DFFEEB0540F196802046082131
:1030A000BDE8F047FFF7D6BED4F890904FF0000887
:1030B0004FF0010AD4F894309B685FFA88F7BB425E
:1030C000FFF451AF09EB4713D3F8002902F4402273
:1030D000B2F5802F24D1D3F80029002A20DAD3F8C2
:1030E000002942F09042C3F80029D3F80029002AB1
:1030F000FBDB3946D4F89000FFF7D6FB22890AFAA9
:1031000007F322EA0303238104EB8703DB689B6850
:1031100013B139462046984739462046FFF780FBD1
:1031200008F10108C6E708EB4112D2F8003B03F4AE
:103130004023B3F5802F10D1D2F8003B002B0CDADE
:10314000628909FA01F322EA0303638104EB810334
:10315000DB68DB680BB12046984701370AE713F0BC
:10316000030F08BF0A68072B98BF027003F1010321
:103170009CBF120A01301EE704EB830301F5805166
:10318000DA6890690268D0F808C04068A2EB000EC7
:1031900000221046974208D1DB689B699A683A443E
:1031A0009A605A6817445F6008E712F0030F08BF7F
:1031B0000868964588BF8CF8000002F1010284BFC0
:1031C000000A0CF1010CE5E7BDE8F08708B50348FB
:1031D000FFF788FEBDE80840FFF776BA8435002087
:1031E00008B50348FFF77EFEBDE80840FFF76CBA5C
:1031F00020360020D0F8903003EB4111D1F8003B8D
:1032000043F40013C1F8003B70470000D0F8903041
:1032100003EB4111D1F8003943F40013C1F8003930
:1032200070470000D0F8903003EB4111D1F8003B1B
:1032300023F40013C1F8003B70470000D0F8903031
:1032400003EB4111D1F8003923F40013C1F8003920
:103250007047000030B5039C0172043304FB032562
:10326000C361049B03630021059B00604060C16053
:10327000426102618561046242628162C1624363AC
:1032800030BD00000022416A41610161C26082627A
:10329000C2626FF00101FEF7D9BE00000369426906
:1032A000934203D1C2680AB100207047181D7047CD
:1032B00003691960C2680132C260C269134482693D
:1032C0000361934224BF436A03610021FEF7B2BE4B
:1032D00038B504460D46E3683BB16269131D1268B8
:1032E000A3621344E362002038BD237A33B9294630
:1032F0002046FEF78FFE0028EDDA38BD6FF00100A2
:10330000FBE70000C368C269013BC3604369134423
:1033100082694361934224BF436A4361002383620D
:10332000036B03B11847704770B52023044683F33D
:103330001188866A3EB9FFF7CBFF054618B186F3C0
:103340001188284670BDA36AE26A13F8015BA36284
:10335000934202D32046FFF7D5FF002383F3118861
:10336000EFE700002DE9F84F04460E4690469946D7
:10337000202787F311880025AA46D4F828B0BBF18E
:10338000000F09D149462046FFF7A2FF20B18BF379
:1033900011882846BDE8F88FA16AE36AA8EB050BFF
:1033A0005B1A9B4528BF9B46BBF1400F1BD9334698
:1033B00001F1400251F8040B43F8040B9142F9D19A
:1033C000A36A40334036A3624035A26AE36A9A4258
:1033D00002D32046FFF796FF8AF311884545D8D2DD
:1033E00087F31188C9E730465A46FDF72FFDA36AD7
:1033F0005B445E44A3625D44E7E7000010B5029CB5
:103400000172043303FB0421C36100238362C3629E
:10341000039B0363049B00604060C46042610261DF
:10342000816104624262436310BD0000026AC260AF
:10343000426A4261026100228262C2626FF001014F
:10344000FEF704BE436902699A4203D1C2680AB119
:1034500000207047184650F8043B0B60704700008E
:10346000C368C2690133C36043691344826943611D
:10347000934224BF436A43610021FEF7DBBD000095
:1034800038B504460D46E3683BB123691A1DA262B4
:10349000E2691344E362002038BD237A33B9294638
:1034A0002046FEF7B7FD0028EDDA38BD6FF00100C9
:1034B000FBE7000003691960C268013AC260C26993
:1034C000134482690361934224BF436A036100236A
:1034D0008362036B03B118477047000070B5202367
:1034E00004460E4683F31188856A35B91146FFF705
:1034F000C7FF10B185F3118870BDA36A1E70A36A5F
:10350000E26A01339342A36204D3E169204604399D
:10351000FFF7D0FF002080F3118870BD2DE9F84F30
:1035200004460D4691469A464FF0200888F31188CC
:103530000026B346A76A4FB951462046FFF7A0FFC1
:1035400020B187F311883046BDE8F88FA06AE76A9A
:10355000A9EB06033F1A9F4228BF1F46402F1BD9E5
:1035600005F1400355F8042B40F8042B9D42F9D196
:10357000A36A4033A3624036A26AE36A9A4204D344
:10358000E16920460439FFF795FF8BF311884E451A
:10359000D9D288F31188CDE729463A46FDF756FC83
:1035A000A36A3B443D44A3623E44E5E702694369A4
:1035B0009A4203D1C3681BB9184670470023FBE742
:1035C000836A002BF8D0043B9B1AF5D01360C368C4
:1035D000013BC360C3691A44836902619A4224BFF4
:1035E000436A0361002383620123E5E700F052B9D7
:1035F000034B002258631A610222DA60704700BF51
:10360000000C0040014B0022DA607047000C0040C3
:10361000014B5863704700BF000C0040FEE70000FC
:1036200010B5194CFEF7FCFBFEF71EFD8022174972
:103630002046FEF7A3FC012344F8180C0374144B36
:10364000144AD96821F4E0610904090C0A431249BB
:10365000DA60CA6842F08072CA60104A1049C2F843
:10366000B01F116841F0010111601022DA772022A9
:1036700083F82220002383F3118862B60948BDE84D
:103680001040FEF79DBC00BF442E00202C400008D7
:1036900000ED00E00003FA05F0ED00E0001000E0AE
:1036A00055CEACC5344000082DE9F84F1F4CDFF86B
:1036B0008090656904F114074FF00008D9F82430B0
:1036C000266AAA689E1B96421DD34FF0200AAA685C
:1036D000236AD5F80CB0134423622B68BB425F60A9
:1036E000A6EB02066361C5F80C8001D1FFF78AFFE3
:1036F00088F311882869D8478AF311886569AB680F
:103700009E42E4D2DAE76269BA420CD09168236241
:103710008E1B9660A86802282CBF1818981CBDE85C
:10372000F84FFFF775BFBDE8F88F00BF1C2E0020D3
:10373000000C0040034B59685A68521A9042FBD85B
:10374000704700BF001000E04B6843608B688360E7
:10375000CB68C3600B6943614B6903628B69436249
:103760000B6803607047000008B52C4B2C48D3F859
:10377000882040F2FF710A43C3F88820D3F88820DC
:1037800022F4FF6222F00702C3F88820D3F88820D1
:10379000D3F8E0200A43C3F8E020D3F808210A4315
:1037A000C3F808211F4AD3F808311146FFF7CCFFB0
:1037B0001D4802F11C01FFF7C7FF1C4802F1380148
:1037C000FFF7C2FF1A4802F15401FFF7BDFF194885
:1037D00002F17001FFF7B8FF174802F18C01FFF703
:1037E000B3FF164802F1A801FFF7AEFF144802F13B
:1037F000C401FFF7A9FF134802F1E001FFF7A4FF9E
:10380000114802F1FC01FFF79FFF104802F58C718F
:10381000FFF79AFFBDE8084000F016B900440258CF
:1038200000000258544000080004025800080258E2
:10383000000C0258001002580014025800180258D8
:10384000001C025800200258002402580028025888
:1038500008B500F0C7FAFFF7E3FEFEF713FFBDE877
:103860000840FEF785BD000070470000084B1A694C
:10387000920710B508D500241C61202383F311881A
:10388000FFF712FF84F31188BDE81040FEF71CBF5C
:10389000000C0040124BD3F8E82042F00802C3F8B5
:1038A000E820D3F8102142F00802C3F810210D4A95
:1038B000D3F81031D36B43F00803D3630A4B632270
:1038C0009A624FF0FF32DA6200229A615A63DA603C
:1038D0005A6001225A6108211A603220FDF76ABC41
:1038E000004402580010005C000C0040F8B5514B39
:1038F000D3F880204FF0FF32C3F880200024D3F8A3
:103900008010C3F88040D3F88010D3F88410C3F837
:103910008420D3F88410C3F88440D3F88410D96F7E
:1039200041F0FF4141F4FF0141F4DF4141F07F01EB
:10393000D967D96F21F0FF4121F4FF0121F4DF4164
:1039400021F07F01D967D96FD3F888106FEA415110
:103950006FEA5151C3F88810D3F88810C1F30A01F7
:10396000C3F88810D3F88810D3F89010C3F89020CB
:10397000D3F89010C3F89040D3F89010D3F8941077
:10398000C3F89420D3F89410C3F89440D3F894105B
:10399000D3F89810C3F89820D3F89810C3F898403B
:1039A000D3F89810D3F88C10C3F88C20D3F88C106F
:1039B000C3F88C40D3F88C10D3F89C10C3F89C202B
:1039C000D3F89C20C3F89C40D3F89C3000F0EAF96F
:1039D000194B07229A60194ADA60194A1A610522BE
:1039E0005A60184A536A43F480335362C2F88440E1
:1039F000BFF34F8FD2F88030C3F3C904C3F34E3303
:103A00005B01A50743F6E07603EA060E2846214649
:103A10004EEA00070139C2F874724F1C00F14040B1
:103A2000F6D1203B13F1200FEED1BFF34F8FBFF340
:103A30006F8FF8BD0044025890ED00E000000430A4
:103A40001B00080300ED00E05A4B5B4901221A609D
:103A50005A4B19609A605A4ADA6000221A614FF490
:103A600040429A619A699204FCD51A6842F48072C5
:103A70001A60544B1A6F12F4407F1FBF4FF480320C
:103A80001A6700221A671A6842F001021A604D4A4A
:103A9000134611684807FCD5002111611A6912F01C
:103AA0003802FBD1012119604FF0804159605A67FB
:103AB000454ADA62454A1A611A6842F480321A604D
:103AC000404A134611688903FCD5116841F0800112
:103AD00011601A68D205FCD53D4A3E499A6200221F
:103AE0005A631963A1F5C0214B39DA6399635A64AB
:103AF000394A1A64394ADA621A6842F0A8521A60DE
:103B0000304B1A6802F02852B2F1285FF9D109222D
:103B10009A610022DA611A624FF00052DA64304989
:103B2000304A1A6559659A652F4A212111601A6930
:103B300042F003021A61234B1A6902F03802182A74
:103B4000FAD1D3F8DC2042F00052C3F8DC20D3F8DD
:103B5000042142F00052C3F80421D3F80421D3F821
:103B6000DC2042F08042C3F8DC20D3F8042142F08C
:103B70008042C3F80421D3F80421D3F8DC2042F0BA
:103B80000042C3F8DC20D3F8042142F00042C3F81D
:103B90000421D3F80421D3F8F42042F00202C3F840
:103BA000F420D3F81C2142F00202C3F81C21D3F800
:103BB0001C3170470881005100C000F000480258D5
:103BC00002000001004402580000FF010088900834
:103BD000222040006302070147040508FD0BFF0196
:103BE0000010E0000000011000200052084A08B553
:103BF000936811680B4003F00103936023B1054AF9
:103C000013680BB150689847BDE80840FEF75CBDEB
:103C100080000058D0380020084A08B59368116821
:103C20000B4003F00203936023B1054A93680BB184
:103C3000D0689847BDE80840FEF746BD80000058B0
:103C4000D0380020084A08B5936811680B4003F08B
:103C50000403936023B1054A13690BB15069984777
:103C6000BDE80840FEF730BD80000058D038002085
:103C7000084A08B5936811680B4003F00803936085
:103C800023B1054A93690BB1D0699847BDE8084054
:103C9000FEF71ABD80000058D0380020084A08B549
:103CA000936811680B4003F01003936023B1054A39
:103CB000136A0BB1506A9847BDE80840FEF704BD8F
:103CC00080000058D0380020174B10B59C681A6847
:103CD000144004F478729A60A30604D5134A936AD8
:103CE0000BB1D06A9847600604D5104A136B0BB12C
:103CF000506B9847210604D50C4A936B0BB1D06BDF
:103D00009847E20504D5094A136C0BB1506C9847EB
:103D1000A30504D5054A936C0BB1D06C9847BDE858
:103D20001040FEF7D1BC00BF80000058D038002002
:103D30001A4B10B59C681A68144004F47C429A60CF
:103D4000620504D5164A136D0BB1506D98472305D3
:103D500004D5134A936D0BB1D06D9847E00404D598
:103D60000F4A136E0BB1506E9847A10404D50C4A4C
:103D7000936E0BB1D06E9847620404D5084A136F56
:103D80000BB1506F9847230404D5054A936F0BB1CC
:103D9000D06F9847BDE81040FEF796BC80000058F1
:103DA000D0380020062108B50846FDF703FA0621A1
:103DB0000720FDF7FFF906210820FDF7FBF9062192
:103DC0000920FDF7F7F906210A20FDF7F3F906218E
:103DD0001720FDF7EFF906212820BDE80840FDF780
:103DE000E9B9000008B5FFF781FD00F00DF8FDF717
:103DF00087FBFDF75FFDFDF731FCFFF735FDBDE803
:103E00000840FFF7F3BB0000002304491A465A504C
:103E1000C8180833802B4260F9D17047D038002091
:103E200010B501390244904201D1002010BD10F8B4
:103E3000013B11F8014FA342F5D0181B10BD000043
:103E4000034611F8012B03F8012B002AF9D1704722
:103E500012101213121100005C2E0020B029002055
:103E600053544D333248373F3F3F3F3F000000003F
:103E700000960000000000000000000000000000AC
:103E8000000000000000000000000000C91400084D
:103E9000B5140008F1140008DD140008E914000846
:103EA000D5140008C1140008AD140008FD14000862
:103EB00000000000D5150008C1150008FD15000818
:103EC000E9150008F5150008E1150008CD150008F2
:103ED000B915000859160008000000000100000094
:103EE00000000000020000000000000001180008AF
:103EF0006D18000840004000F43200200433002018
:103F000002000000000000000300000000000000AC
:103F1000B118000800000000100000001433002059
:103F200000000000010000000000000084350020B7
:103F30000101020025424F415244250025534552BC
:103F400049414C25005069786861776B3600303103
:103F50003233343536373839414243444546000020
:103F6000486F6C7962726F005069786861776B3660
:103F70002D424C0011230008852100086D17000810
:103F8000F5220008430000008C3F000809024300AE
:103F9000020100C0320904000001020201000524F0
:103FA000001001052401000104240202052406007A
:103FB00001070582030800FF09040100020A00004E
:103FC00000070501024000000705810240000000D3
:103FD00012000000D83F000812011001020000404A
:103FE00062314B00000201020301000004030904D6
:103FF00000000000211A0008011D0008AD1D000886
:1040000040004000BC360020BC360020010000000B
:10401000CC360020800000004001000008000000B5
:104020000001000000040000080000006D61696EDE
:10403000000000004C400008D8360020D038002096
:10404000010000001D3600080000000069646C6576
:10405000000000000000802A00000000AAAAAAAA0E
:1040600000000000FFFF00000000000000A00A00A8
:104070000400000000000000AAAAAAAA0000000094
:10408000FDFF0000000000000000000000500000E4
:1040900000000000AAAAAAAA000000003FFF00003A
:1040A0000000000000000000000000000000000010
:1040B000AAAAAAAA00000000FFFF0000000000005A
:1040C000000000000000020000000000AAAAAAAA46
:1040D00000000100FFFF00000000000007000000DA
:1040E0000020000000000000AAAAAAAA00100000F8
:1040F000FFFF0000000000070000000000000000BB
:1041000000000000AAAAAAAA00000000FFFF000009
:10411000000000000000000000000000000000009F
:10412000AAAAAAAA00000000FFFF000000000000E9
:10413000000000000000000000000000AAAAAAAAD7
:1041400000000000FFFF0000000000000000000071
:104150000000000000000000AAAAAAAA00000000B7
:10416000FFFF000000000000000000000000000051
:1041700000000000AAAAAAAA00000000FFFF000099
:104180000000000000000000FF0000000000000030
:10419000603E00083F00000000960000000008009C
:1041A00004000000EC3F00080000000000000000D8
:1041B00000000000000000000000000000000000FF
:00000001FF
